:020000040000FA
:04000000B5EF01F067
:080008000D6E240E056EF40ECE
:10001000066EA5D8D8B4CA94D8A4CA84FC0FD8A0B8
:10002000CA92D8B0CA82056A240E066EF40E096E12
:100030000A6ACAB425D8CAB223D893D80504CB6EAD
:1000400005C007F006C008F000500B6E0C6E003CB7
:100050000C6A9CD80A500D2E0AD0BE6E0C0EBD6ED6
:1000600009BEBD8A09BCBD889494CA841200BB6EC7
:100070000C0EBA6E09BEBA8A09BCBA889492F5D73A
:1000800000D8D8900932063205321200080E03B4A7
:10009000010E086E076A0F0EEA6E00C0E9FF0150FC
:1000A00085D80150EF120C0E4CD8015000C0E9FF6A
:1000B000EF14FF0F03A4073203B407363C0E41D8F8
:1000C000082EEDD70750D8801200076E080E03B433
:1000D000010E086E0F0EEA6E00C0E9FF015066D8EF
:1000E0000000000001500732D8B0EF123C0E29D8B2
:1000F0000150EF12082EF0D7D880120003A2120090
:1001000003D0036E03A012000F0EEA6E00C0E9FFD9
:1001100001504CD8010E066EF40E14D80150EF12A7
:10012000010E066EF40E0ED0086A076EFF0E07264B
:10013000082200D0D8A01200030E066EE60E02D8E8
:10014000F5D7066AFE0F056E000000D000D0E86A01
:10015000065AD8A01200050600D000D0F5D70A6ACA
:10016000096A100EF36E063409360A360750095C28
:1001700008500A5805E30750095E08500A5AD8800B
:1001800005360636F32EEFD70550120007500B0246
:10019000F3CF09F0F4CF0AF008500B02F3500A260F
:1001A00007500C02F3500A2609501200FF0AEF16FE
:1001B00000D0E988E92AEC161200165012181D6EBC
:1001C0001DBE34D016BE19D01550115CD8A0000C3D
:1001D000D8A4010C1650125CD8A0000CD8A4010CB5
:1001E0001750135CD8A0000CD8A4010C1850145C54
:1001F000D8A0000CD8A4010C000C1150155CD8A09C
:10020000000CD8A4010C1250165CD8A0000CD8A485
:10021000010C1350175CD8A0000CD8A4010C14508A
:10022000185CD8A0000CD8A4010C000C12AE010C74
:10023000000C1250106E16181E6E1150D8A41550D6
:100240003CE011267E0E03E3115E03E338D0115E1D
:1002500033E314C00EF013C00FF0108E168E146A24
:10026000136A126A180E1C6E10320F320E3206E339
:10027000185014261750132216501222123213321D
:1002800014321C2EF1D712BE07D014361336123694
:10029000115212E0110610341BAC17D016E3143EB5
:1002A00014D0133E12D0123E10D0D8801232133226
:1002B0001432113E0AD003D01B84116A02D01B8273
:1002C0001168146A136A800E126E1EAE129E1450CC
:1002D0001200136A146A960E1C6E1E9E14AE07D08E
:1002E000D880000E11561256135614561E8E1452F4
:1002F00018E01BAC0DD014AE0BD0122A09E1132A62
:1003000007E1142A05E1D8801432133212321C2A74
:10031000080E1C2612C011F013C012F014C013F006
:1003200011D013520FE1080E1C5E125007E1080EA7
:100330001C5E115002E1145010D0116A136E11C0EE
:1003400012F0116A13BE06D0D89011361236133649
:100350001C06F8D71EAE139E1C5011C014F0116E6F
:10036000135012C013F0126E1200F86A400E1B6E8A
:10037000AB6AAC6A7B6A7A6A7E6A7F6AC26AA66A7C
:10038000A68E280E006E980E076E3A0E086E010EAD
:100390003BDE00D0820E006E010E016E036EB1DEF8
:1003A000CC0E93DE440E91DE190EBEDE820E006E80
:1003B000010E016E036A6ADE07C021F02150046E4F
:1003C0000452F2E0820E006E010E016E036E99DEA1
:1003D000CC0E7BDEBE0E79DE820E006E010E016E4B
:1003E000020E036E53DE1F6E51DE206E4FDE07C01D
:1003F00021F04CDE07C021F049DE07C021F046DEC7
:1004000007C021F043DE07C021F040DE07C022F024
:1004100075DE1FC011F020C012F05BDF186A176A8A
:10042000166A7B0E156E05DF14C026F013C025F08A
:1004300012C024F011C023F024BE09D0000E265CA7
:10044000000E2558440E2458840E23580AE2280E24
:10045000006E980E076E3A0E086E010E04EC00F066
:10046000C7D0660E146E136E440E126E840E116E9B
:1004700026C018F025C017F024C016F023C015F0D0
:100480009CDE01081BE026C014F025C013F024C038
:1004900012F023C011F0186A176A480E166E840E07
:1004A000156E8BDE01080AE04B0E006E980E076E8B
:1004B0003A0E086E010E04EC00F09AD0660E146E2F
:1004C000136E480E126E840E116E26C018F025C0F1
:1004D00017F024C016F023C015F06FDE01081BE0F2
:1004E00026C014F025C013F024C012F023C011F070
:1004F000186A176A4C0E166E840E156E5EDE0108C1
:100500000AE0640E006E980E076E3A0E086E010E39
:1005100004EC00F06DD0660E146E136E4C0E126E6D
:10052000840E116E26C018F025C017F024C016F0F6
:1005300023C015F042DE01081BE026C014F025C0E0
:1005400013F024C012F023C011F0186A176A500E7D
:10055000166E840E156E31DE01080AE07D0E006E07
:10056000980E076E3A0E086E010E04EC00F040D0B3
:10057000660E146E136E500E126E840E116E26C02F
:1005800018F025C017F024C016F023C015F015DEB2
:1005900001081BE026C014F025C013F024C012F09F
:1005A00023C011F0186A176A540E166E840E156E69
:1005B00004DE01080AE0C80E006E980E076E3A0EBF
:1005C000086E010E04EC00F013D024BE11D0010E11
:1005D000265C000E2558540E2458840E235808E338
:1005E0000068980E076E3A0E086E010E04EC00F0DB
:0A05F000190E94EC00F0CED6FFD7F0
:020000040030CA
:0300010006190ECF
:020005008180F8
:060008000FC00FE00F40E5
:00000001FF
